:020000020000FC
:10000000DFEFDDBF00240EBE2AC00810022008204A
:100010000100042000200408020002080120021050
:1000200000004FB735EC51B1587F05BA503D10F480
:10003000503608F43061503839F463B16D1708F068
:100040006D2F6ABD68BD63BD583A11F4C3B935EC74
:10005000583B11F4D3B935E836BF4FBF189508E0C7
:10006000102E10BE00E40ABD08BD03BD08EB01BBA5
:1000700001EA0FBD01E00EBD01E605BD02BA14BAEA
:1000800015BA00EC08BB0A95F1F708E5B79B0250DA
:10009000B69B045002E502B9789405EC06BFEAE08D
:1000A000F0E026E0AFEF80E12A95CAF3059107BBA7
:1000B000059102BB00BE06EE07B903ED06B9349BFD
:1000C000FECF05B1000F000FC01708F4C3950C1741
:1000D00008F4CA95C13448F0C23818F00ABC08BC0C
:1000E00003BCDD2321F0DA9502C0D395E1F306B815
:1000F00010BE059107B91591BB27FF2408B1007206
:10010000011739F400E1B00F08F4BFEFAB2F80E125
:10011000CBCFFA9499F7B395BA1781F78A9521F660
:02012000C1CF4D
:00000001FF
